:100000000C949E000C9429110C94BB000C94BB0022
:100010000C94BB000C94BB000C94BB000C94BB0074
:100020000C94BB000C94BB000C94BB000C94BB0064
:100030000C94BB000C94BB000C94BB000C94BB0054
:100040000C94BB000C94BB000C94BB000C94BB0044
:100050000C94BB000C94BB000C94BB000C94BB0034
:100060000C94BB000C94BB00240352006500740088
:1000700072006F0020004100640061007000740095
:100080006500720020004D006F006400090222002C
:1000900001010080FA0904000001030000000921A9
:1000A000010100012250000705810308000412012C
:1000B0001001000000080D0FC10001040102000141
:1000C00005010905A101150025013500450175014E
:1000D000950E05091901290E81029502810105017C
:1000E0002507463B01750495016514093981426570
:1000F000009501810126FF0046FF00093009310902
:10010000320935750895048102750895018101C091
:10011000FF00020104FF03FF0607FFFF05FFFFFFCB
:10012000FFFF00020104FF03FF0607FFFF050403B2
:1001300009040A034D006F004A006F0011241FBE1E
:10014000CFEFD4E0DEBFCDBF11E0A0E0B1E0E8E941
:10015000F4E202C005900D92A230B107D9F711E088
:10016000A2E0B1E001C01D92AF34B107E1F70E94F7
:100170005C030C944A120C9400000F931F93FF939E
:10018000EF93BF93AF93F92FE82F09E0009310018D
:1001900000E20093110100E00093120101E00093DE
:1001A000130101E00093140100E000931501009396
:1001B00016010093170109E20093180107D0BF91BF
:1001C000AF91EF91FF911F910F910895A1E0B0E1E0
:1001D00009E02D980000000000002C9800000000AD
:1001E00000002C9A000000002C9800000000000085
:1001F0002C9A0000000000002C9800000000000075
:100200002C9A0000000000002C9800000000000064
:100210002C9A00000000000000002D9A1D9117FD8F
:100220002C9A17FF2C982D98000000002C9A16FD90
:100230002D9A16FF2D982C9A000000002D9A15FD7E
:100240002C9A15FF2C982D9A000000002C9A14FD72
:100250002D9A14FF2D982C9A000000002D9A15FD60
:100260002C9A15FF2C982D9A000000002C9A14FD52
:100270002D9A14FF2D982C9A000000002D9A15FD40
:100280002C9A15FF2C982D9A000000002C9A14FD32
:100290002D9A14FF2D982C9A000000002D9A0A9593
:1002A0002D9A2C9A0895F92FE82FCF93DF93D72F0B
:1002B000C62F21E030E0E20FF31F22273327442727
:1002C0005527662777278827992790E099D0B6D0B9
:1002D00082D0292F80D0392F7ED0492F253031F080
:1002E0002930A1F180E0DF91CF910895BFEFBA9559
:1002F000F1F7B8ECBA95F1F791E082D09FD06BD0CE
:10030000292F69D0392F67D0492F65D0592F4083C5
:10031000518340E050E027FD426026FD416025FD0D
:10032000546024FD52602F7035FD406434FD4068F8
:1003300033FD486032FD446031FD406130FD406274
:1003400045835683822FDF91CF910895B4E6BA9505
:10035000F1F790E455D093E053D092E051D06ED0B5
:100360003AD0292F38D0392F36D0492F34D0592FB1
:1003700032D0692F30D0792F2ED0892F2CD04058F1
:10038000505840835183605870586283738340E0B3
:1003900050E020FD426021FD416022FD486023FDC8
:1003A000446024FD526034FD546035FD406836FDE4
:1003B000406436FF8C8335FF9D83458356833F70B1
:1003C000232F3E7F31FD31603D7F20FD3260832F42
:1003D000DF91CF91089590E0B4E1A8E0BA9579F06B
:1003E0001899FCCFB9E0BA95F1F7990F1899916077
:1003F000B4E1BA9521F0189BFCCFAA9579F708953E
:10040000A8E097FD0DC0209ABDE0BA95F1F7000075
:100410002098B3E0BA95F1F7990FAA9591F708954E
:10042000209AB3E0BA95F1F7000000002098BDE0F3
:10043000BA95F1F7990FAA9521F70895209AB3E09C
:10044000BA95F1F700000000209808951AB889EFD6
:100450008BB914B88FE385B917B888B90895FC0132
:10046000808180768032E1F48181813041F482E0C4
:1004700091E0909334018093330188E008958230B5
:1004800041F48FE091E0909334018093330181E057
:1004900008958A3029F4838180930F0180E00895C4
:1004A00080E00895CF92DF92EF92FF920F931F9317
:1004B000CF93DF93FC01DB01E80187018081805845
:1004C00080838C9180588C93DA018C9180588C9326
:1004D000F901808180588083D601EC91EE2341F0B0
:1004E000F0E0EF70F070E05FFE4FE491EC9303C03A
:1004F0008FEFF60180832881D8013C91832F822BD6
:1005000009F444C018821C92922F20FF03C08881F6
:100510008260888391FF03C088818460888392FF12
:1005200003C088818160888393FF03C088818860CD
:10053000888394FF03C088818064888395FF03C00B
:1005400088818068888396FF03C088818061888362
:1005500022231CF4888180628883932F30FF04C09B
:10056000F80180818160808391FF04C0D8018C9163
:1005700082608C9392FF04C0F80180818460808344
:1005800093FF04C0D8018C9188608C93DF91CF9148
:100590001F910F91FF90EF90DF90CF900895682FFB
:1005A000F894E2E0F1E088E0DF011D928A95E9F736
:1005B000359959C0349950C086B190E08E719070D1
:1005C0008430910511F18530910534F4009771F074
:1005D000029709F054C00FC08830910501F18A30AC
:1005E0009105C1F0069709F04AC00AC082E091E087
:1005F0000E94660D5AC082E091E00E94FE0B55C039
:1006000082E091E00E94CB0650C082E091E00E941F
:100610008D0738C082E091E00E945E0646C083B13B
:1006200090E0867090708230910589F08630910557
:1006300021F0892B39F081E023C082E091E00E9413
:10064000B50533C082E091E00E9447052EC082E0EC
:1006500091E00E94B90729C0339914C082E091E06B
:100660000E94210F22C0339905C082E091E00E94D0
:100670002C041BC082E091E00E94B30803C080E01C
:10068000882399F489B1897061F44C9B05C082E09C
:1006900091E00E94BF0309C082E091E00E94AC0A91
:1006A00004C082E091E00E940208E8E6F0E0808168
:1006B0008E7F8083789408952F923F924F925F921D
:1006C0006F927F928F929F92AF92BF92CF92DF9262
:1006D000EF92FF920F931F93DF93CF9300D000D040
:1006E000CDB7DEB70E9426020E94960F0F2EF4E2CD
:1006F000AF2EF1E0BF2EF02D85E091E001969A83B8
:1007000089830F2EF5E02F2EF1E03F2EF02DE2E051
:10071000F0E02E0E3F1E0F2EF5E04F2EF1E05F2E83
:10072000F02D83E090E0480E591EE5E0F1E03397AC
:10073000FC83EB833F010894611C711C882499247D
:10074000689481F88E0E9F1E0E94A80FF50180818B
:1007500084FFFACF81E00E94CF0285E091E06981B9
:100760007A81A10192010B811C81730164010E94B5
:1007700052028B819C8168E00E94E610E5CF0F93C6
:100780001F93DF93CF93CDB7DEB728970FB6F894BA
:10079000DEBF0FBECDBF8C01E5E2F0E080818E7F31
:1007A0008083E4E2F0E080818E7F8083EBE2F0E002
:1007B00080818F778083EAE2F0E0808180688083A7
:1007C000FE01319688E0DF011D928A95E9F7C801A4
:1007D000BF010E945301282F83FF04C0F8018281CA
:1007E0008160828322FF07C0D80112968C911297F4
:1007F000846012968C9321FF04C0F8018281886086
:10080000828320FF07C0D80112968C9112978260D4
:1008100012968C93F80184818195848386818195D9
:10082000868328960FB6F894DEBF0FBECDBFCF915A
:10083000DF911F910F910895E4E2F0E02081277F7E
:100840002083208120632083E5E2F0E0208128637B
:1008500020830E94BD000895DC01EAE2F0E080817F
:100860008E7E8083EBE2F0E0808181618083E4E230
:10087000F0E080818863808380818D7F8083E5E2E2
:10088000F0E0808182608083E7E2F0E08081807E1A
:100890008083E8E2F0E080818F618083489B0BC019
:1008A000E4E2F0E0808184608083E5E2F0E0808132
:1008B000837C808314C0E4E2F0E080818B7F8083BE
:1008C000E5E2F0E080818C638083E7E2F0E0808104
:1008D0008E7F8083E8E2F0E080818160808387E121
:1008E00080937E00EAE7F0E085E0808384E68093F1
:1008F0007C00808180688083808186FDFDCF6130AF
:1009000009F5EAE7F0E0808180648083808186FDDC
:10091000FDCF909179008FE7891B14968C931497E3
:1009200082E680937C00EAE7F0E080818064808347
:10093000808186FDFDCF909179008FE7891B13960A
:100940008C931397E9E2F0E0808110927A00109284
:100950007E00808180FF10C04C9905C0613019F481
:100960008C9181608C93199975C0623009F072C0C6
:100970008C9181608C930895E5E2F0E08081877F1F
:10098000808385E08A95F1F7309903C08C9182606D
:100990008C931A9903C08C9180618C93199903C030
:1009A0008C9180688C934C9907C011968C9111970B
:1009B000846011968C931197E5E2F0E08081886065
:1009C000808380818F7E808385E08A95F1F73099DE
:1009D00003C08C9184608C931A9903C08C918062BF
:1009E0008C93199907C011968C911197816011967B
:1009F0008C9311974C9903C08C9181608C93E5E2A4
:100A0000F0E080818061808380818F7D808385E0BC
:100A10008A95F1F7309903C08C9188608C931A996C
:100A200003C08C9180648C93199907C011968C91A6
:100A30001197826011968C9311974C9906C011966C
:100A40008C911197886011968C93E5E2F0E080819B
:100A500080628083089590E020E0A3E2B0E0EBE2C2
:100A6000F0E035E1220F8C9180FD216080818F774D
:100A70008083832F8A95F1F7808180688083832F1C
:100A80008A95F1F79F5F983069F7822F0895CF9389
:100A9000DF93EC01ABE2B0E08C91886F8C938C918A
:100AA0008E7F8C93EAE2F0E08081896C8083808184
:100AB0008F7C8083E4E2F0E080818E7F8083E5E2BA
:100AC000F0E08081816080838C918F7B8C930E9489
:100AD0002B05282F30E0C901807F9070803491056C
:100AE00009F040C020FF03C08A8188608A8321FF0B
:100AF00003C08A8182608A8322FF03C08A81816069
:100B00008A8323FF03C08A8184608A830E942B0525
:100B1000282F982F81FF03C088818064888392FFEB
:100B200003C088818068888393FF03C089818160C6
:100B3000898394FF03C089818260898395FF03C004
:100B400088818460888396FF03C08881826088835F
:100B500022231CF4888181608883EBE2F0E08081AD
:100B600080648083DF91CF910895DC01EAE2F0E0B8
:100B7000808186708083EBE2F0E08081896F8083E2
:100B8000E4E2F0E08081807C8083E5E2F0E0808137
:100B90008F638083E9E2F0E08081982F91708081FB
:100BA00083FD926080910B01981709F466C0913023
:100BB000F1F0913038F0923009F441C0933009F0EF
:100BC00051C029C0813041F412968C9112978260F5
:100BD00012968C93129746C0823009F043C0129649
:100BE0008C911297886012968C9312973BC0833039
:100BF00041F412968C911297826012968C93129700
:100C000031C0882379F512968C91129788601296DC
:100C10008C93129727C0823041F412968C911297D0
:100C2000826012968C9312971DC08130D9F412966F
:100C30008C911297886012968C93129713C0882318
:100C400041F412968C911297826012968C931297AF
:100C500009C0833039F412968C91129788601296ED
:100C60008C93129790930B0183E080930A01129664
:100C70008C91129780930C010CC080910A018823FB
:100C800041F0815080930A0180910C0112968C935F
:100C900012974E9903C08C9181608C930895EBE27A
:100CA000F0E080818F7E80838CE291E00197F1F704
:100CB00089B190819061908381700895CF93DF9383
:100CC000EC01E4E2F0E08081837C808380818260BB
:100CD0008083A5E2B0E08C918E638C93EAE2F0E031
:100CE00080818E7F8083808180618083EBE2F0E071
:100CF0008081816180838C918D7F8C931D9903C04D
:100D00008A8181608A831C9903C08A8184608A8376
:100D10001B9903C08A8188608A831A9903C08A81DB
:100D200082608A830E944F06882319F4888182603A
:100D300088830E944F06882319F488818160888304
:100D40000E944F06882319F48881886088830E9456
:100D50004F06882319F48881846088830E944F0697
:100D6000882319F48881806888830E944F0688232D
:100D700019F48881806488830E944F06882319F4BF
:100D8000898182608983E5E2F0E0808182608083EE
:100D9000DF91CF910895CF93DF93DC01E4E2F0E09F
:100DA0008081837C8083808182608083E5E2F0E0C3
:100DB00080818E638083EAE2F0E0808180618083BD
:100DC000EBE2F0E080818F7E808392E02BE230E0E6
:100DD000E3E2F0E045E250E0E90188818F7E88831C
:100DE0000000000080818C7309F44FC0808185FD74
:100DF00007C012968C911297816012968C9312976D
:100E0000808184FD07C012968C91129782601296A1
:100E10008C931297808183FD07C012968C91129754
:100E2000846012968C931297808182FD07C012967F
:100E30008C911297886012968C931297EA018881A0
:100E40008D7F888300000000808185FD03C08C9128
:100E500082608C93808184FD03C08C9181608C932F
:100E6000808183FD07C011968C9111978160119646
:100E70008C931197808182FD26C011968C911197D9
:100E8000826011968C9311971EC0EA0188818D7F34
:100E9000888300000000808185FD03C08C91846000
:100EA0008C93808184FD03C08C9188608C938081B9
:100EB00083FD03C08C9180648C93808182FD03C08C
:100EC0008C9180688C93E901888180618883EA0134
:100ED000888182608883915009F07ECFDF91CF9125
:100EE000089590E020E0E5E2F0E03AE6A3E2B0E029
:100EF00080818B7F8083832F8A95F1F726958C9153
:100F000085FD2068808184608083832F8A95F1F736
:100F10009F5F983069F7822F0895EF92FF920F93A9
:100F20001F937C0105E210E0F80180818C7E8083B4
:100F3000808184628083E4E2F0E080818F7D808321
:100F400080818C618083F80180818860808388EC57
:100F500090E00197F1F70E947107F8018081877F87
:100F600080838AEAF70181831F910F91FF90EF90B0
:100F70000895DC01EAE2F0E0808186708083EBE294
:100F8000F0E08081896F8083E4E2F0E080818E7FF1
:100F90008083E5E2F0E08081816080834E9908C023
:100FA0008C9181608C9304C09F5F9B3F21F40895D6
:100FB00090E0E3E2F0E0808180FDF6CF89B1982FE8
:100FC000892F8095282F217093FF226094FF246041
:100FD00095FF286090E0E3E2F0E003C09F5F9B3F55
:100FE00081F0808180FFFACF89B180FF206183FF8B
:100FF000206284FF206485FF20688FE7821B1396A0
:101000008C930895DC01EAE2F0E0808186788083A9
:10101000808180688083EBE2F0E080818F7780833D
:10102000808189678083E4E2F0E080818E7F808325
:10103000E5E2F0E08081816080838AE48A95F1F7BF
:1010400089B1807311F090E011C04E9903C08C916A
:1010500081608C93189B02C091E008C011968C911E
:101060001197826011968C93119791E0EBE2F0E07A
:101070008081806880838AE48A95F1F7489907C067
:1010800012968C911297816012968C9312974B99BD
:1010900007C012968C911297846012968C931297C7
:1010A0004C9907C012968C911297886012968C9377
:1010B00012974D9907C012968C91129782601296E2
:1010C0008C931297992359F44E9903C08C918160A7
:1010D0008C93189942C08C9182608C933EC04E993B
:1010E00003C08C9182608C93189903C08C918460AA
:1010F0008C93EBE2F0E080818F7780839AE4892FF4
:101100008A95F1F7808180688083892F8A95F1F72D
:1011100080818F7780839A95F1F789B18973E9F49B
:101120008081806880838AE48A95F1F7489903C0BA
:101130008C9180688C934B9903C08C9180648C93C4
:101140004C9903C08C9188608C934D9906C0119680
:101150008C911197816011968C93EBE2F0E0808185
:10116000806880830895DC01E4E2F0E08081817C86
:101170008083E5E2F0E080818E638083E7E2F0E047
:101180008081807C8083E8E2F0E080818F638083CF
:10119000EAE2F0E080818E7E8083EBE2F0E0808105
:1011A000816180831D9907C011968C911197816090
:1011B00011968C9311971C9903C08C9188608C9325
:1011C0001B9903C08C9182608C931A9907C0129668
:1011D0008C911297826012968C931297199907C07E
:1011E00012968C911297846012968C931297329972
:1011F00007C011968C911197826011968C9311976C
:10120000319903C08C9184608C93309903C08C9188
:1012100081608C930895DC018AE48A95F1F783B1AB
:101220008C7011F090E011C0199903C08C9181600D
:101230008C93319B02C091E008C011968C9111975C
:10124000826011968C93119791E0E8E2F0E0808142
:10125000846080838AE48A95F1F71D9904C080E850
:1012600014968C9314971C9904C08FE714968C9352
:1012700014971B9904C080E813968C9313971A99BE
:1012800004C08FE713968C931397992359F41999F7
:1012900003C08C9181608C93319942C08C918260A3
:1012A0008C930895199903C08C9182608C93319925
:1012B00003C08C9184608C93E8E2F0E080818B7FA6
:1012C00080839AE4892F8A95F1F7808184608083F6
:1012D000892F8A95F1F780818B7F80839A95F1F72A
:1012E00083B18C73E9F48081846080838AE48A9579
:1012F000F1F71D9903C08C9180688C931C9903C0F1
:101300008C9180648C931B9903C08C9188608C9322
:101310001A9906C011968C911197816011968C9341
:10132000089583B1E8E2F0E090819D7F908320E80A
:10133000922F9A95F1F79081926090832A95F1F718
:1013400086958695809581700895CF93DF93EC0103
:10135000E4E2F0E080818B7F8083E5E2F0E0808151
:1013600084608083E7E2F0E0808184608083A8E28B
:10137000B0E08C9184608C938081826080838C91BA
:1013800082608C9380EC90E00197F1F78C918B7FD9
:101390008C9380E88A95F1F70E949109882319F0CF
:1013A0008881826088830E949109882319F088814E
:1013B000816088830E949109882319F08981816066
:1013C00089830E949109882319F089818260898329
:1013D0000E949109882311F080E88C830E94910972
:1013E000882311F08FE78C830E949109882311F0E4
:1013F00080E88B830E949109882311F08FE78B830B
:101400000E949109882319F08881846088830E9452
:101410009109882319F08881886088830E94910946
:10142000882319F08881806488830E949109882329
:1014300019F08881806888830E949109882321F0AF
:1014400088818370888319C08881282F207F288312
:10145000982F80FF03C0822F8460888391FF03C090
:1014600088818160888392FF03C08881826088833D
:1014700093FF03C0888188608883DF91CF910895AE
:101480009C01E4E2F0E08081817C8083E5E2F0E091
:1014900080818E638083E7E2F0E0808184608083D6
:1014A00080818D7F8083E8E2F0E0808182608083AC
:1014B00080818B7F808383B1887321F4C9010E946E
:1014C000A5090895C9010E940B090895282F2695A2
:1014D00011F437E009C037E0982F990F822F8170FF
:1014E000892B31502695C1F790E002C0880F991FD3
:1014F0003A95E2F7089589B1E5E2F0E090819E7FA8
:10150000908320E8922F9A95F1F7908191609083D3
:101510002A95F1F782958695877080958170089558
:1015200020E090E0A9E2B0E0E5E2F0E030E82695C6
:101530008C9185FF206880818E7F8083832F8A95A0
:10154000F1F7808181608083832F8A95F1F79F5F17
:10155000983069F7822F08950F931F93CF93DF93ED
:10156000EC01EAE2F0E080818F7D8083ABE2B0E0C5
:101570008C9180628C938081806880838C9180685C
:101580008C93E4E2F0E0808181608083E5E2F0E02A
:1015900080818160808380EC90E00197F1F78C91ED
:1015A0008F778C9380E88A95F1F70E94900A182F24
:1015B0000E94900A082F0E94900A982F11231CF471
:1015C0008A8182608A83212F30E016FF03C08A81DE
:1015D00088608A8325FF03C08A8184608A8324FF10
:1015E00003C08A8181608A83F901E870F07023FF6B
:1015F00003C0898182608983B9016470707022FFA1
:1016000003C0898181608983892F8F70883009F0B8
:101610005AC0812F82958F70982F80FF03C08A81D6
:1016200081608A8391FF03C08A8184608A8392FFEC
:1016300003C08A8188608A8393FF03C08A818260A5
:101640008A83802F8095482F4F70483008F0405192
:10165000842F90E0880F991F880F991F909581958E
:101660009F4F8C83802F90E080959095807F907025
:101670009595879595958795959587959595879552
:10168000482F883008F04051842F90E0880F991F30
:10169000880F991F909581959F4F8B83EF2B19F0A1
:1016A000898182608983672B19F0898181608983B0
:1016B00021FF03C088818160888320FF6CC08881FE
:1016C0008260888368C0402F50E0CA01807C90709F
:1016D000803C9105D1F50F3F21F081E080930D0111
:1016E0000FC080910D01882359F421FF03C0888128
:1016F0008160888320FF4FC08881826088834BC0CF
:1017000020FF02C08FE78E8321FF02C080E88D8317
:1017100040FF02C08FE78D8341FF02C080E88E83C7
:1017200042FF03C088818064888343FF03C08881AF
:101730008068888344FF03C088818160888345FF77
:101740002AC088818260888326C0802F807F09F527
:1017500010920D0121FF03C088818460888320FFDF
:1017600003C088818160888340FF03C088818260D4
:10177000888341FF03C088818860888342FF03C05B
:1017800088818064888343FF06C08881806888835D
:1017900002C010920D01DF91CF911F910F9108951A
:1017A000382F80E18A95F1F790E020E0E5E2F0E063
:1017B00040E4A3E2B0E030FF04C080818061808318
:1017C00003C080818F7E808380818B7F8083842F84
:1017D0008A95F1F726958081846080838C9185FDC0
:1017E0002068842F8A95F1F79F5F983011F0369525
:1017F000E2CF80E18A95F1F7822F0895DF92EF9290
:10180000FF920F931F93CF93DF93EC01E4E2F0E09C
:1018100080818D7D808380818C618083E5E2F0E032
:1018200080818E6380838081877F808380E18A9539
:10183000F1F781E00E94D00B82E40E94D00B082FC8
:1018400010E0813409F411E0DD24033711F4DD24C4
:10185000D394EE24FF24093719F4EE24FF24E394F3
:1018600080E090E0033511F481E090E09701282BAF
:10187000392B812F8D2990E0282B392B232B09F42C
:1018800086C08FEF0E94D00B8FEF0E94D00B282FC5
:10189000982F80FD03C089818160898393FD03C0F7
:1018A0008981826089831123A9F094FD03C08A8114
:1018B00081608A8396FD03C08A8184608A832223A3
:1018C0001CF08A8188608A8395FD16C08A818260B7
:1018D0008A8312C0DD2081F091FD03C0898184607C
:1018E000898392FD03C0898188608983822F8295D4
:1018F0008F7080958F708A838FEF0E94D00B282F76
:10190000982F80FD03C088818061888391FD03C08A
:1019100088818062888392FD03C088818064888387
:1019200093FD03C088818068888394FD03C088810B
:101930008860888395FD03C088818260888396FDD6
:1019400003C088818160888322231CF088818460A1
:10195000888380E0033509F481E08D2990E08E29A9
:101960009F29892BA1F08FEF0E94D00B80588D8387
:101970008FEF0E94D00B80588E838FEF0E94D00B88
:1019800080588B838FEF0E94D00B80588C8303325A
:1019900009F04AC08FEF0E94D00B8FEF0E94D00B4E
:1019A000982F83FD03C0898182608983892F829566
:1019B0008F7080958F708A838FEF0E94D00B282FB5
:1019C00083FD03C088818068888324FD03C08881EB
:1019D0008860888325FD03C08881826088838FEFBB
:1019E0000E94D00B80588B838FEF0E94D00B282F42
:1019F000813838F080E890E0821B9109880F991FA8
:101A00008E838FEF0E94D00B882334F090E08058B3
:101A10009F4F880F991F8E838FEF0E94D00B8138C4
:101A200018F0888180648883E5E2F0E08081886036
:101A3000808380E18A95F1F7DF91CF911F910F911B
:101A4000FF90EF90DF900895EF92FF920F931F9316
:101A5000CF93DF937C01E5E2F0E08081877F808394
:101A6000062F10E01016110664F4C0E0D0E0F70174
:101A7000EC0FFD1F80810E94D00B2196C017D1076B
:101A8000B4F3E5E2F0E080818860808380E18A95AC
:101A9000F1F7DF91CF911F910F91FF90EF90089593
:101AA00090E0E3E2F0E003C09F5F983C19F0808192
:101AB00081FDFACF089590E0E3E2F0E003C09F5F7C
:101AC000983C19F0808181FFFACF08950F931F93FE
:101AD000CF93DF93EC01E4E2F0E080818D7C8083A2
:101AE00080818C608083E5E2F0E080818E6380837A
:101AF000EAE2F0E080818E7E8083EBE2F0E080819C
:101B0000816180838AE08A95F1F7489B5BC04C999C
:101B100003C0888180618883E5E2F0E08081877F6F
:101B200080838AE08A95F1F71C9903C08A818160DD
:101B30008A831D9903C08A8184608A83489903C07F
:101B40008A8188608A834C9903C08A8182608A83F3
:101B5000E5E2F0E08081837F886080838AE08A9577
:101B6000F1F71C9903C08881826088831D9903C0A6
:101B7000888184608883489903C0888181608883D4
:101B80004C9903C0898182608983E5E2F0E080811D
:101B9000837F80838AE08A95F1F71C9903C088814E
:101BA000806888831D9903C08881806488834899F0
:101BB00003C08881886088834C993EC18881806297
:101BC00088833AC11C9B38C1E5E2F0E08081877FC1
:101BD000808380818B7F80830E94500D1C991BC164
:101BE00005E210E0F8018081846080830E945B0D33
:101BF000F80180818B7F80830E94500D1C9903C067
:101C00008A8181608A831D9903C08A8184608A8366
:101C1000489903C08A8188608A834C9B02C010E087
:101C20001AC08A8182608A8310E015C08A8181602F
:101C30008A831D9903C08A8184608A83489903C07E
:101C40008A8188608A834C9B02C011E004C08A812B
:101C500082608A8311E0E5E2F0E080818460808325
:101C60000E945B0D1C9903C08881826088831D9946
:101C700003C0888184608883489903C0888181601B
:101C800088834C9903C0898182608983E5E2F0E012
:101C900080818B7F80830E94500D1C9903C08881B6
:101CA000806888831D9903C08881806488834899EF
:101CB00003C08881886088834C9903C088818062D2
:101CC0008883E5E2F0E08081846080830E945B0D80
:101CD0004C9903C0888180618883E5E2F0E08081CF
:101CE0008B7F80830E94500D1C9902C000E101C0CF
:101CF00000E01D9B0062489B00644C9B0068E5E28D
:101D0000F0E08081846080830E945B0D1C9B0160F9
:101D10001D9B0260489B04604C9B0860113019F4C5
:101D20008FE7801B8B83E5E2F0E080818B7F8083EF
:101D30000E94500D1C9902C000E101C000E01D9BF3
:101D40000062489B00644C9B0068E5E2F0E0808103
:101D5000846080830E945B0D1C9B01601D9B026060
:101D6000489B04604C9B0860113019F48FE7801B7E
:101D70008C83E5E2F0E080818B7F80830E94500DB0
:101D80001C9902C000E101C000E01D9B0062489B5D
:101D900000644C9B0068E5E2F0E080818460808311
:101DA0000E945B0D1C9B01601D9B0260489B0460B0
:101DB0004C9B0860113019F4802F86958E83E5E2E4
:101DC000F0E080818B7F80830E94500D1C9902C0BF
:101DD00000E101C000E01D9B0062489B00644C9B39
:101DE0000068E5E2F0E08081846080830E945B0D02
:101DF0001C9B01601D9B0260489B04604C9B08601B
:101E0000113019F4802F86958D83E5E2F0E0808112
:101E10008C60808311C005E210E0F801808184604D
:101E200080830E945B0DF80180818B7F80830E94FC
:101E3000500D1C9BFBCEFDCEDF91CF911F910F91DA
:101E40000895DC01E4E2F0E08081817C8083E5E2BA
:101E5000F0E080818E638083E7E2F0E08081827C25
:101E60008083808182608083E8E2F0E080818F63FC
:101E7000808380818D7F808380818260808390E8F1
:101E800020E1E3E2F0E0822F8A95F1F7808185FF7F
:101E900003C013969C931397808184FF03C014960C
:101EA0009C931497808183FF03C015969C9315978C
:101EB000808182FF03C016969C9316979F5F9F3781
:101EC00011F713968C9113978E3719F413961C9271
:101ED000139714968C9114978E3719F414961C92BC
:101EE000149715968C9115978E3719F415961C92A8
:101EF000159716968C9116978E3719F416961C9294
:101F00001697309903C08C9181608C93199903C006
:101F10008C9182608C934C9903C08C9184608C93DB
:101F2000489903C08C9188608C930895E9E6F0E0AD
:101F3000808182608083EDE3F0E080818160808336
:101F4000E5E2F1E08BE4808331978AE580830895B0
:101F50001F93CF93DF9380913501982F93500AF40C
:101F6000B6C020913201809131018D3209F0ADC0AF
:101F7000983009F0AAC08CE090E0821B9109FC0126
:101F8000E75CFE4FEF0183EC809319018AE58093B3
:101F9000000110920E018081807629F0CF010E940D
:101FA0002F02982F89C0928110922201818188236B
:101FB00031F4E3E2F1E0108292E0319779C08530AC
:101FC00031F49093360190E0E2E2F1E071C08630A6
:101FD00009F04EC08381813041F48EEA90E0909305
:101FE00034018093330192E13FC0823041F48CE8A8
:101FF00090E0909334018093330192E235C08330B6
:10200000F1F4992341F48EE291E0909334018093AE
:10201000330194E029C0913041F482E391E0909340
:102020003401809333019AE01FC09230E1F488E6D6
:1020300090E0909334018093330192E115C0813296
:1020400041F48EE990E0909334018093330199E05C
:102050000BC0823241F480EC90E090933401809385
:10206000330190E501C090E080E480930E0124C02C
:10207000883021F491E0E8E3F1E01AC0893031F4CE
:102080009093380190E0E2E2F1E012C08A3021F44E
:1020900091E0E2E2F1E00CC08B3021F090E0E2E26E
:1020A000F1E006C08BE48093250190E0E2E2F1E0EC
:1020B000F0933401E09333018F81882321F48E81E2
:1020C000891708F4982F909301011092350180919F
:1020D000000184FF57C0109101011F3F09F452C055
:1020E000193008F05CC010920101E9E1F1E0808153
:1020F00098E889278083112309F45DC0209133017A
:102100003091340180910E0186FF14C0AAE1B1E044
:1021100080E090E0F901E80FF91FE491ED9301965A
:102120001817C1F7812F815090E00196F901E80F4F
:10213000F91F0FC0D901912FEAE1F1E08D91819350
:102140009150E1F7812F815090E00196F901E80F5D
:10215000F91FF0933401E0933301193068F48AE1F8
:1021600091E0612F0E942511612F6C5F6C3040F46B
:102170008FEF8093010104C08FEF809301016EE126
:102180006093000194E1E9E2F0E080818670D1F48F
:102190009150D9F7109236011092300113C0812F5F
:1021A000885080930101E9E1F1E0808198E8892776
:1021B000808318E0A3CF8AE191E060E00E942511BE
:1021C00064E0D6CFDF91CF911F910895FF920F93D6
:1021D0001F93DC01F62E8091240184FF07C0E5E205
:1021E000F1E0808198E88927808303C08AE58093A5
:1021F00024019F2DE6E2F1E08D9181939150E1F76A
:1022000006E211E0C8016F2D0E9425118F2D8C5F11
:1022100002501040F80180831F910F91FF900895A4
:10222000A82FB92F80E090E041E050EA609530E0BF
:1022300009C02D9182279795879510F084279527BF
:10224000305EC8F36F5FA8F30895EADF8D939D9326
:102250000895CF93CFB7CF93DF93C395499BE9F709
:10226000499B0BC0499B09C0499B07C0499B05C0BE
:10227000499B03C0499B01C08BC06F93C091320141
:10228000DD27C75CDE4F2F9365E5499B03C02F9187
:102290006F91E6CF0F931F934F9320E040E15F9340
:1022A00009B1067001FB27F93F9350E03BE039C0CC
:1022B000167040642F77012F5F5F1EC0406819B110
:1022C00016702F7752501FC0406409B12F770670E7
:1022D000D1F15F5F00C023C0406219B12F77167043
:1022E00091F15F5F00C025C006701027515012F4B5
:1022F0005D5F0000115027952C3F19B1C8F616708C
:102300000127015027952C3FC8F64227499309B170
:10231000067010274F73115027952C3FA8F646954D
:10232000469519B1167079F00127015027952C3F79
:1023300098F66B5A60F3315009B1B0F600C011E065
:102340001CBB002719C03B503195C31BD04011E086
:102350001CBB0881033C09F10B34F9F020913001DA
:102360001981110F1213EDCF4A81441F093651F123
:102370000D3211F0013E29F7009337013F915F9133
:102380004F911F910F912F916F91CCB3C0FD65CFED
:10239000DF91CF91CFBFCF911895209137012223A4
:1023A00069F310913501112391F5343092F1309396
:1023B000350120933101109132013BE0311B309304
:1023C000320127C00091350101300CF50AE54F704C
:1023D00049F43091000134FD1DC000930001C9E1B2
:1023E000D1E01CC03091240134FD14C000932401BD
:1023F000C5E2D1E013C0052710E000C000000BB912
:102400001AC0052710E0221F1DC010E021C04AE5B8
:1024100002C032ED432FC4E1D0E032E01AB11660C1
:10242000599A0BB11AB956E020E865E320FF052759
:102430000BB9279517951C3FF0F66695B8F7B1F7DD
:1024400020FF05270BB9279517951C3FD0F6279538
:10245000179517FF052700001C3F0BB9B0F629910F
:102460003A9519F7097F10913601110FC651D040E6
:102470000BB911F01093300111E01CBB02601AB1CE
:10248000197F402F497F54E05A95F1F70BB91AB9DB
:082490004BB974CFF894FFCFA3
:022498005AFFE9
:00000001FF
